:100000000C9489000C94A6000C94A6000C94A600F5
:100010000C94A6000C94A6000C94A6000C94A600C8
:100020000C94A6000C94A6000C94A6000C94A600B8
:100030000C94A6000C94A6000C94A6000C9419082D
:100040000C94A6000C94A6000C94A6000C94A60098
:100050000C94A6000C94A6000C94A6000C94A60088
:100060000C94A6000C94A6000C94A6000C94A60078
:100070000C94A6000C94A6000C94A6000C94A60068
:100080000C94A6000C94A6000C94A60049324320C0
:10009000535441525420434F4E444954494F4E20EB
:1000A0004552524F520049324320534C415645204D
:1000B00041444452455353204552524F5200493215
:1000C000432044415441205458204552524F52003D
:1000D0004932432044415441205258204552524F06
:1000E00052004932432054494D454F55540049323E
:1000F00043204552524F520A0020545743523D2547
:10010000303278205354415455533D253032780ACB
:10011000000011241FBECFEFD0E1DEBFCDBF11E044
:10012000A0E0B1E0ECE3FBE100E00BBF02C0079010
:100130000D92A836B107D9F711E0A8E6B1E001C0E9
:100140001D92A437B107E1F70C947A080C940000D3
:100150002F923F924F925F926F927F928F929F92D7
:10016000AF92BF92CF92DF92EF92FF920F931F93C5
:10017000CF93DF93CDB7DEB726970FB6F894DEBFE7
:100180000FBECDBF5C016A017B01522E180127FF13
:1001900002C0552405C085E2821714F485E2582E6A
:1001A000D5019896BE83AD8320E030E040E050E07A
:1001B000C701B6010E94D70B882354F4F101808156
:1001C0009181826091838083F7FAF094F7F8F0943C
:1001D000AE014F5F5F4FC701B6010E94370C3B0174
:1001E0004C01E980FA800B811C8120E030E040E086
:1001F00050E0C801B7010E94D70B8823E9F1CD80F8
:10020000DE80442428C02DEC3CEC4CEC5DE3C801BE
:10021000B7010E94670CAE014F5F5F4F0E94370C21
:100220002AE939E941E251E40E94670C0E94BC0BC3
:10023000605DD6016E936D014394E980FA800B8175
:100240001C8120E030E040E050E0C801B7010E948E
:10025000D70B882319F0AC14BD04A8F2750106C0B1
:10026000F60181916F01D7018D937D01ED81FE81B2
:10027000CE16DF06A8F329C020E030E040E050E0D1
:10028000C401B3010E94DA0B18161CF07501442456
:100290001CC0442403C04A943701480120E030E0E8
:1002A00040E251E4C401B3010E94670C7B018C0160
:1002B00020E030E040E85FE30E94D70B87FDEBCF02
:1002C000E982FA820B831C837501D1014D915C9107
:1002D00053FF13C0BDEF4B1684F0242D332727FDA9
:1002E0003095852D992787FD909501962817390718
:1002F00024F45460F10151834083D1018D919C918C
:1003000092FD08C05394052D112707FD10950A0D85
:100310001B1D0CC0052D112707FD10950A0D1B1D77
:10032000842D992787FD9095080F191F0A151B0525
:10033000D8F4F5014CC020E030E040E251E4C401C3
:10034000B3010E94670CAE014F5F5F4F0E94370CF4
:100350003B014C0169817A818B819C810E94BC0B9D
:10036000605DD7016D937D010E151F0528F0ED81AD
:10037000FE81EE16FF06F8F28D819E81081719079F
:1003800018F0F50117A224C0D8018C918B5F8C93D3
:10039000F80131E318C020E3D8012C93A016B10670
:1003A00028F48E918D018F5F8C930DC0D8013C9302
:1003B0004394D1018D919C9192FF05C0AE16BF066A
:1003C00008F420833196D8018C918A3324F7108267
:1003D000842D992787FD909526960FB6F894DEBF59
:1003E0000FBECDBFDF91CF911F910F91FF90EF9086
:1003F000DF90CF90BF90AF909F908F907F906F9045
:100400005F904F903F902F9008952F923F924F9280
:100410005F926F927F928F929F92AF92BF92CF9294
:10042000DF92EF92FF920F931F93CF93DF93CDB79D
:10043000DEB7EE970FB6F894DEBF0FBECDBFCC246B
:10044000DD2476013C017EAF6DAF5A011A8219821C
:10045000FC0117821682838181FDF3C38FEF9FEF2A
:1004600016C409811A8100FFD3C3842D80538A30BA
:10047000D0F4F0E34F1631F4552021F403FD02C00F
:10048000116075C18AE0252D2802C0011124542C69
:10049000580E30ED530E57FE02C04FE7542E03FDA9
:1004A000CAC3352CC8C3442D45564CAF433028F041
:1004B000842D8554833008F0FCC0C501049698AFA4
:1004C0008FABF501C080D180E280F38003FD02C0D4
:1004D00036E0532E077B1A83098346015701A70193
:1004E0009601C701B6010E94B3088823C1F08EE4CB
:1004F0008D838B8381E48C839E012A5F3F4F3AAFCB
:1005000029AF3CAD333008F07AC28B81805E8B839B
:100510008C81805E8C838D81805E8D8370C2C701EB
:10052000B6010E942E0C892BE9F089E48D838EE4BC
:100530008C8386E48B8320E030E040E050E0C7010C
:10054000B6010E94D70B87FD06C0AE014A5F5F4F20
:100550005AAF49AFD6CF8DE28E83CE0107969AAFC0
:1005600089AFCFCFC80192609A838983E7E44E16A2
:1005700009F449C0E41544F0F5E44F1679F026E497
:10058000421609F042C31DC036E64316D1F047E6D5
:100590004416C9F155E6451609F037C38E010F5FC1
:1005A0001F4F252DB501A401CE010F960E94A80072
:1005B000282E8CEF380E15140CF43A94DE011F9699
:1005C00015C094609A8389838E010F5F1F4F252D7C
:1005D000B501A401CE010F960E94A800282E151483
:1005E0000CF43A94DE011F96121444F4FD010190BC
:1005F0000020E9F73197CE2ECA1A02C0C52CC39449
:10060000BAAFA9AF7DC1552011F0252D01C021E061
:1006100098609A8389838E010F5F1F4FB501A401F3
:10062000CE010F960E94A800282E89819A8192FF00
:100630001EC0822D850D8150282FA82FBB27A7FD16
:10064000B095AC0FBD1F1F9605C08C91119721501E
:10065000803331F4622F27FD23C02215B4F703C382
:10066000C62E562E5218539400C3C92E17C0252DDE
:10067000E52DFF27E7FDF095EC0FFD1F3F9606C027
:1006800080813197292F2150803379F7922F1216CC
:10069000BCF3522EC22E222309F4EFC2592EEDC212
:1006A000E22FFF27E7FDF095EC0FFD1F108A552480
:1006B00099CFC8018870907003FF04C0552011F4D1
:1006C00021E0522EE9E64E1609F493C0E4153CF100
:1006D000F3E54F1609F474C0F415ACF02BE24216A2
:1006E000E1F1241544F030E24316D1F143E244161F
:1006F00009F080C23FC05DE24516C1F18EE24816A6
:1007000009F078C239C093E64916E1F1E4E64E16E5
:1007100009F46FC0F8E54F1609F06CC29FC020E7DE
:10072000421609F496C0241544F03CE6431641F104
:100730004FE6441609F05EC20DC055E7451609F4B0
:100740008FC0E8E74E1609F489C0F3E74F1609F0A9
:1007500051C221C028E02BAF83C000611A830983F6
:1007600089819A8180629A83898365C200681A832D
:10077000098361C20064FBCF08601A83098352C2F7
:100780000460F5CFA5014E5F5F4F58AF4FABF50149
:10079000C0803A9434C1F501C080D180892B41F0EA
:1007A000652D772767FD7095C6010E94960918C0D0
:1007B000F60101900020E9F73197EC19EBAF11C079
:1007C000F501C080D180892B41F0652D772767FD29
:1007D0007095C6010E948B0903C0C6010E94820960
:1007E0008BAF95012E5F3F4F38AF2FAB3BAD331A28
:1007F00006C102FF0BC0A5014C5F5F4F58AF4FAB66
:10080000F50160817181828193810EC095012E5F17
:100810003F4F38AF2FABF501808191819C01B90129
:10082000882777FD8095982F6B017C0197FF0BC07F
:1008300002601A830983F094E094D094C094C11CA0
:10084000D11CE11CF11C89819A818F7B9A83898359
:1008500027C000641A83098398E7492E30E13BAF33
:1008600029813A8122FF0BC0A5014C5F5F4F58AF31
:100870004FABF50160817181828193810CC0A5012C
:100880004E5F5F4F58AF4FABF50180819181AC0156
:10089000BA01882799276B017C012F7C3A83298331
:1008A00087017601CE0103969AAF89AF9BADA92E41
:1008B000BB24CC24DD24C801B701A60195010E9408
:1008C000310D6A301CF0640D615201C0605DE9AD0C
:1008D000FAAD6193FAAFE9AFC801B701A60195017E
:1008E0000E94310D79018A0121153105410551051B
:1008F00011F7CC24DD247601CE010396C9ACC81AC9
:1009000049815A81CA0182739070892B09F03A9407
:1009100046FF07C0FBADF03111F482E001C081E079
:10092000381A43FF10C0252D332727FD30958C2D15
:1009300099278217930724F0477F5A83498303C07E
:100940005C18351801C03C1840785170452B69F48B
:10095000832D06C0B30180E290E00E94F109812F4F
:10096000182F11501816B4F3312E89819A8181FF06
:1009700004C0B3018DE290E00BC084FF04C0B3015A
:100980008BE290E005C085FF05C0B30180E290E0F6
:100990000E94F10989819A8186FF0FC0B30180E32B
:1009A00090E00E94F1092BAD203139F4B301842D80
:1009B000992787FD90950E94F10989819A8190FF7E
:1009C0000DC0832D06C0B30180E390E00E94F109C1
:1009D000812F182F11501816B4F3312E89819A8166
:1009E00083FF0DC0252D06C0B30180E390E00E9477
:1009F000F109212F122F11501216B4F3512E8981B3
:100A000087FD0DC0832D06C0B30180E290E00E94F7
:100A1000F109812F182F11501816B4F3312E33E637
:100A2000431631F4B3018C2D992787FD9095BEC0F4
:100A300043E74416B1F4460156011BAD09C0F50168
:100A400081915F01B301992787FD90950E94F1097B
:100A50001150A8F76401FBADCF0ED11C2FEF2BAFC7
:100A6000B8C033E54316B1F446018601BBAC08C0FB
:100A7000F8018491B30199270E94F1090F5F1F4F7C
:100A8000BA94FFEFBF16A1F764012BADC20ED11CC3
:100A9000FBAF9FC089819A8191FD03C009AD1AAD5A
:100AA00091C092FF1DC01214BCF4A9ACBAAC122DB7
:100AB00009C0F50181915F01B301992787FD9095E8
:100AC0000E94F1091150A8F729AD3AAD220D311D50
:100AD0003AAF29AF22240FC0B30180E390E009C0F0
:100AE000E9ADFAAD8191FAAFE9AFB301992787FD7E
:100AF00090950E94F10915142CF4B3018EE290E058
:100B00000E94F10989819A8192FD06C017C0B30144
:100B100080E390E00E94F1092394822D815087FFA9
:100B20000DC05A94852D8F5F18168CF307C0B30142
:100B3000892F992787FD90950E94F109E9ADFAADBB
:100B40009191FAAFE9AF992329F05A94852D8F5FDF
:100B500018166CF389819A8192FD3BC0B301842DF4
:100B6000992787FD90950E94F1092A9427FE07C0D6
:100B7000B3018DE290E00E94F109219405C0B30118
:100B80008BE290E00E94F1096AE070E0822D9927E3
:100B900087FD90950E941E0D6B017C01CB01C096D4
:100BA000B3010E94F109B301C701C0960E94F10987
:100BB00010C0F80182918F01B301992787FD9095AC
:100BC0000E94F109CE0103960817190791F71AAF91
:100BD00009AF898187FF17C0832D06C0B30180E26A
:100BE00090E00E94F109812F182F11501816B4F3CC
:100BF000312E09C0B301842D992787FD90950E945D
:100C0000F109B8AEAFAA1A821982AFA8B8AC13C066
:100C1000F5E24F1649F481E090E09A8389832AE057
:100C20002BAF3324552407C0B301842D992787FDAA
:100C300090950E94F1094DAD5EAD4F5F5F4F5EAF85
:100C40004DAFF301838183FF04C0EDADFEAD449051
:100C500003C0EDADFEAD4080442009F002CCF301AD
:100C60008681978114C0C22E5524EC2DFF27E7FD05
:100C7000F095EC0FFD1F108AB2CCEC2DFF27E7FD9D
:100C8000F095EC0FFD1F108AFEEF4F0E92CCEE9602
:100C90000FB6F894DEBF0FBECDBFDF91CF911F918D
:100CA0000F91FF90EF90DF90CF90BF90AF909F900B
:100CB0008F907F906F905F904F903F902F9008950E
:100CC00084E980937400E4E7F0E0808184FDFDCF47
:100CD00080E090E00895CF92DF92EF92FF920F9321
:100CE0001F936C01E62E042F0E946006DF92CF92C4
:100CF0000E943E0A11271F930F93FF24FF92EF9249
:100D000089EF90E09F938F930E943E0A8DB79EB724
:100D100008960FB6F8949EBF0FBE8DBF1F910F911E
:100D2000FF90EF90DF90CF900895EF92FF920F9396
:100D30001F93FC01342F522F109269011092680109
:100D4000662321F084EC8093740003C084E88093D0
:100D500074008091740088233CF080916801909128
:100D60006901885E9340A8F38091680190916901C0
:100D7000885E9340E0F05523B1F10F2EF1E7EF2E9E
:100D8000FF24F02DF701408104E710E0F8016081B5
:100D900080ED90E00E946B06F7014081F8016081D0
:100DA00082EE90E00E946B068FEF9FEF1EC0409195
:100DB0007100842F9927887F9070232F3327821703
:100DC000930759F0552379F06091740080ED90E01D
:100DD0000E946B068FEF9FEF08C0809173008083A5
:100DE00080E090E002C08FEF9FEF1F910F91FF9086
:100DF000EF900895EF92FF920F931F93542F10924C
:100E00006901109268018093730084E880937400F4
:100E1000E4E7F0E0808188233CF0809168019091C4
:100E20006901885E9340B0F38091680190916901F7
:100E3000885E9340E0F0552399F10F2EF1E7EF2EF5
:100E4000FF24F02DF701408104E710E0F8016081F4
:100E50008EEB90E00E946B06F7014081F801608103
:100E600082EE90E00E946B068FEF9FEF1BC04091D7
:100E70007100842F9927887F9070262F332782173F
:100E8000930719F480E090E00DC0552349F060917C
:100E900074008EEB90E00E946B068FEF9FEF02C014
:100EA0008FEF9FEF1F910F91FF90EF900895EF92BA
:100EB000FF920F931F93342F522F109269011092BB
:100EC0006801880F862B8093730084E880937400F8
:100ED000E4E7F0E0808188233CF080916801909104
:100EE0006901885E9340B0F3809168019091690137
:100EF000885E9340E0F0552399F10F2EF1E7EF2E35
:100F0000FF24F02DF701408104E710E0F801608133
:100F100086EA90E00E946B06F7014081F80160814B
:100F200082EE90E00E946B068FEF9FEF1BC0409116
:100F30007100842F9927887F9070232F3327821781
:100F4000930719F480E090E00DC0552349F06091BB
:100F5000740086EA90E00E946B068FEF9FEF02C05C
:100F60008FEF9FEF1F910F91FF90EF900895EF92F9
:100F7000FF920F931F93282F10926901109268011E
:100F800084EA80937400E4E7F0E0808188233CF0F9
:100F90008091680190916901885E9340B0F38091DF
:100FA000680190916901885E9340E0F0662361F1E9
:100FB0000F2EF1E7EF2EFF24F02DF701408104E71B
:100FC00010E0F80160818CE890E00E946B06F70168
:100FD0004081F801608182EE90E00E946B068FEF05
:100FE0009FEF14C040917100421719F480E090E027
:100FF0000DC0662349F0609174008CE890E00E9477
:101000006B068FEF9FEF02C08FEF9FEF1F910F9145
:10101000FF90EF9008959C0112BE1092690110920A
:101020006801809168019091690182179307C9F75F
:1010300008951F920F920FB60F9211248F939F93D2
:101040008091680190916901019690936901809364
:1010500068019F918F910F900FBE0F901F90189570
:1010600013BE86B7836086BF87B7836087BF8DE076
:1010700083BF12BE83E781BF08955D9BFECF8CB90D
:1010800080E090E008951F93CF93DF9310E0C1E0DC
:10109000D0E0C09A8AE090E00E940B0861E088E00E
:1010A0000E94B707882301F520E048E160E08C2F1B
:1010B0000E945707882369F4DF93CF9380E091E083
:1010C0009F938F930E941E0A1F5F0F900F900F90A7
:1010D0000F900E946006C0988AE090E00E940B0882
:1010E0002196CF37D105A9F6812F9927DF91CF918E
:1010F0001F910895CFEFD0E1DEBFCDBF0E94300831
:10110000B89A109290008FE589B988E08AB97894EE
:1011100060E070E08DE398E00E94A109E1E7F0E073
:1011200080818C7F80838CE180937000E4E7F0E025
:1011300080818460808380E291E00E946D0A0E9439
:10114000430899279F938F9380E491E09F938F9317
:101150000E941E0A83E591E00E946D0A0F900F9095
:101160000F900F90FFCFA8E1B0E0E9EBF8E00C940E
:10117000770D69837A838B839C832D833E834F8392
:101180005887BE01675F7F4FCE0101960E94E3083A
:10119000BE016F5E7F4FCE0105960E94E3088985F0
:1011A000823018F481E090E00AC020E030E08989C4
:1011B000823010F0C90103C021E030E0C901E2E053
:1011C00068960C94930DFC01DB01208131819281A2
:1011D000492F4F7750E0991F9927991F8381682FD6
:1011E000660F692B881F8827881FFD01818366236E
:1011F00009F049C0211531054105510509F470C0B8
:1012000082E89FEFFD0193838283220F331F441FE7
:10121000551F220F331F441F551F220F331F441F1A
:10122000551F220F331F441F551F220F331F441F0A
:10123000551F220F331F441F551F220F331F441FFA
:10124000551F83E08C932030F0E03F07F0E04F071C
:10125000F0E45F0790F482E89FEF220F331F441FF2
:10126000551F0197203060E0360760E0460760E4D4
:10127000560798F3FD0193838283FD012483358310
:101280004683578308956F3F71F1862F99278F57B3
:101290009040FD019383828383E08C93220F331F60
:1012A000441F551F220F331F441F551F220F331F8A
:1012B000441F551F220F331F441F551F220F331F7A
:1012C000441F551F220F331F441F551F220F331F6A
:1012D000441F551F506424833583468357830895E4
:1012E00082E08C930895211531054105510519F4CB
:1012F00084E08C93089544FD02C01C92BECF81E02F
:101300008C93BBCFFC0105900020E9F78095909568
:101310008E0F9F1F0895FC010590615070400110D1
:10132000D8F7809590958E0F9F1F0895FC0161500E
:10133000704001900110D8F7809590958E0F9F1FF7
:101340000895EF92FF920F931F93CF93DF938C0139
:101350007B01892B11F4672BD1F16EE070E081E005
:1013600090E00E94A00AFC01009789F1DC0180E86E
:101370008383E114F10471F0F386E28681E88383CC
:1013800080916A0190916B01892B21F4F0936B019C
:10139000E0936A0101151105E1F01187008783814F
:1013A0008260838380916C0190916D01892B89F417
:1013B000F0936D01E0936C0180916E0190916F014B
:1013C000892B39F4F0936F01E0936E0102C0A0E025
:1013D000B0E0CD01DF91CF911F910F91FF90EF9081
:1013E00008950F931F93CF93DF938C01EB018B81B3
:1013F000992781FF1BC082FF0DC02E813F818C8108
:101400009D812817390764F4E881F9810193F983F4
:10141000E88306C0E885F985802F0995892B31F48A
:101420008E819F8101969F838E8302C00FEF1FEFF5
:10143000C801DF91CF911F910F910895CF93DF9352
:10144000CDB7DEB722970FB6F894DEBF0FBECDBF83
:10145000FE01379661917191FA83E983AF01809122
:101460006C0190916D010E94050222960FB6F894CE
:10147000DEBF0FBECDBFDF91CF910895CF93DF9335
:10148000CDB7DEB722970FB6F894DEBF0FBECDBF43
:10149000FE01379661917191FA83E983E0916C01C5
:1014A000F0916D0183818860838349815A818091A5
:1014B0006C0190916D010E940502E0916C01F09128
:1014C0006D012381277F238322960FB6F894DEBF18
:1014D0000FBECDBFDF91CF9108950F931F93CF9390
:1014E000DF938C01E0916C01F0916D01838181FFAC
:1014F0001FC0C0E0D0E00AC0FD0120853185BD01DC
:10150000F9010995892B11F0CFEFDFEFF8018191F7
:101510008F01A0916C01B0916D01882369F7FD01E5
:1015200020853185BD018AE0F9010995892B11F0EB
:10153000CFEFDFEFCE01DF91CF911F910F91089593
:101540000F931F93CF93DF93869F8001879F100D8A
:10155000969F100D1124C8010E94BC0AEC0100974F
:1015600029F0A80160E070E00E94B50BCE01DF9188
:10157000CF911F910F910895CF93DF93AC01029704
:1015800010F442E050E0A0917201B0917301FD01AE
:10159000C0E0D0E020E030E020C08081918184175D
:1015A000950769F482819381209719F09B838A8340
:1015B00004C09093730180937201CF0132C0481729
:1015C000590738F42115310519F08217930708F4EB
:1015D0009C01EF010280F381E02D3097F1F6211597
:1015E000310589F1C901841B950B049708F4A90101
:1015F000E0E0F0E026C08D919C911197821793074F
:10160000E9F44817590779F4ED018A819B813097F5
:1016100019F09383828304C09093730180937201C5
:10162000CD01029649C0841B950BFD01E80FF91FFF
:101630004193519302978D939C933AC0FD01A281EF
:10164000B3811097C1F68091700190917101892B3F
:1016500041F48091630190916401909371018093B2
:10166000700120916501309166012115310541F429
:101670002DB73EB78091610190916201281B390B13
:10168000E0917001F09171012E1B3F0B241735077B
:1016900088F0CA0102962817390760F0CF01840F3D
:1016A000951F02969093710180937001419351931D
:1016B000CF0102C080E090E0DF91CF910895CF93F9
:1016C000DF93009709F44EC0EC0122971B821A8227
:1016D000A0917201B0917301109711F140E050E0B8
:1016E00001C0DC01AC17BD0700F1BB83AA83FE017A
:1016F00021913191E20FF31FEA17FB0771F42E5F7E
:101700003F4F8D919C911197820F931F99838883EE
:10171000FD01828193819B838A834115510559F490
:10172000D0937301C09372011DC0FD01828193812A
:10173000AD010097B1F6FA01D383C28321913191B3
:10174000E20FF31FEC17FD0769F42E5F3F4F88810E
:101750009981820F931FFA01918380838A819B81F3
:1017600093838283DF91CF910895DC0101C06D9353
:1017700041505040E0F7089597FB47D09F3738F02D
:10178000FEE9F91B982F872F762F6B2F05C05AC0C3
:101790009695879577956795F150D0F73EF490959B
:1017A0008095709561957F4F8F4F9F4F08950ED014
:1017B0005EF004C00BD026F001C008D019F020F470
:1017C0008FEF089580E0089581E0089597FB092E3A
:1017D000052600F8689410D0E89407FC07C062174B
:1017E00073078407950721F008F4009407949894F0
:1017F0000895052E092607FA440F551F5F3F79F01B
:10180000AA27A51708F051E04795880F991F9F3F19
:1018100031F0BB27B91708F091E0879508959F91A3
:101820009F91112408C197FB880F991F9F3F31F0AA
:10183000BB27B91708F091E0879508959F919F9174
:101840001124F9C0662777278827992708959F3F95
:1018500059F4803C49F481E09927089590688923E0
:10186000872386238395B9F3882799270895DBDF9B
:10187000CF93DF93D52FC42F552744273327222713
:101880009923D9F09F37C8F0F92FBDD0592F482F91
:10189000372F262FF63968F46FDFA6D0C030CD077A
:1018A00021F069937993899399939058DF91CF911F
:1018B00057C09927882777276627C030CD0721F0A2
:1018C0002993399349935993DF91CF919CC091DF2C
:1018D00001D099C0992339F0552329F09F575F57BC
:1018E000950F13F49AF1B1CF91589F3FE1F3629FA6
:1018F000A12D0F92BB27639FA00DB11DEE27729FF4
:10190000A00DB11DEE1FAF93AA27649FB00DE11D7E
:10191000739FB00DE11DAA1F6627829FB00DE11DC8
:10192000A61F5527749FE00DA11D551F839FE00D35
:10193000A11D561F849FA00D511D852F7A2F6E2F3C
:101940001F900F9088231AF4939539F474C0000CFB
:10195000111CBB1F661F771F881F01280895505850
:10196000192E47DF01D04FC0BA17620773078407EB
:101970009507B1F188F40EF410940B2EBA2FA02D18
:10198000062E622F202D072E732F302D082E842F28
:10199000402D092E952F502DFF275523B9F0591BA7
:1019A00049F0573E98F0469537952795A795F04012
:1019B0005395C9F776F0BA0F621F731F841F30F476
:1019C000879577956795B795F040939517FA0F2E01
:1019D0000895BF1BBB27BA0B620B730B840BF6CFAA
:1019E000DEF633CFE89403C097FB0EF4D8DEB62FB3
:1019F000672F782F892F9EE9002405C09A95BB0F89
:101A0000661F771F881F11249923A1F08823B2F73E
:101A10009F3F59F0BB0F48F421F4002011F460FF00
:101A200004C06F5F7F4F8F4F9F4F881F979587959B
:101A300097F9089507CF9FEF80EC089597FB092E43
:101A400007260AD077FD04D02ED006D000201AF445
:101A5000709561957F4F0895F6F7909581959F4F0A
:101A60000895A1E21A2EAA1BBB1BFD010DC0AA1FDF
:101A7000BB1FEE1FFF1FA217B307E407F50720F0F7
:101A8000A21BB30BE40BF50B661F771F881F991F72
:101A90001A9469F760957095809590959B01AC01BB
:101AA000BD01CF010895AA1BBB1B51E107C0AA1FAE
:101AB000BB1FA617B70710F0A61BB70B881F991FEF
:101AC0005A95A9F780959095BC01CD0108952F9264
:101AD0003F924F925F926F927F928F929F92AF92BE
:101AE000BF92CF92DF92EF92FF920F931F93CF930B
:101AF000DF93CDB7DEB7CA1BDB0B0FB6F894DEBFA2
:101B00000FBECDBF09942A88398848885F846E84C7
:101B10007D848C849B84AA84B984C884DF80EE8011
:101B2000FD800C811B81AA81B981CE0FD11D0FB61A
:0C1B3000F894DEBF0FBECDBFED0108959C
:101B3C00666F756E642064657669636520617420D8
:101B4C0061646472657373203078253032780A00D2
:101B5C000A0A49324320627573207363616E6E65A5
:101B6C0072207374617274696E67202E2E2E0A00B7
:101B7C000A2575206465766963657320666F756EDA
:101B8C00640A007363616E20636F6D706C657465BD
:081B9C000020007401000000AC
:00000001FF
